:020000040000FA
:0600000060283D300130D4
:08000800A000030EA100831209
:100010008B1C2E288B1031181328B11C2E2864300D
:100020000102031C2D281428152816281728182823
:1000300019281A281B283110B114A810031005190B
:100040000314AA0DA90DA80DB00B2E2831152A08EE
:10005000AF002908AE002808AD00B11081010B11D6
:0A006000210E8300A00E200E0900FF
:1000C000203084008001840A80300402031C6228EE
:1000D0001230B0007B2283160C3085058701831215
:1000E000850187010730990000309A00103083168F
:1000F0008E008312603083168F00831200308316C7
:1001000091009F008312C830831681008312313022
:100110009000003083168C00831210308B00BD1BC2
:100120009328851DC4223D1BBE013D1BBF013D1F01
:10013000B92281018E018F010B118B100B108C01E4
:100140008B17B2203119C8204D22B30BAF280310F2
:1001500085190314BA0DF0303A020319A321BD1812
:10016000EC22A1286400311808000B1D08000B11B7
:10017000B11031141230B000051DC328321483169B
:10018000011383120800321083160117831208002E
:10019000321CCF282D090339AD00AE09AF09E43078
:1001A0002F02F0300319AF004C302F020C3003192E
:1001B000AF006C302F023C300319AF00EC302F023F
:1001C000FC300319AF00B3302F02F3300319AF0036
:1001D0001B302F020F300319AF003B302F023F308E
:1001E0000319AF00BB302F02FF300319AF003111EC
:1001F0000130B7008B132030370783169B001C1487
:100200001A088312A400A5002510103037078316A2
:100210009B001C141A088312A300003037078316B2
:100220009B001C141A088312A2008B1722082D02AF
:10023000031D9D2923082E06FC39031D9D2901302D
:1002400003303702031D482900302E060339031DF1
:100250002D29BF1F3629BF13B11703302E060339CE
:10026000031D3629BF1B3629BF17B11744302F068F
:100270005439031D3F293F1F08003F13B1171030A9
:100280002F065439031D48293F1B08003F17B1179B
:10029000AF13AF12AF11AF1024082F02031D742942
:1002A00001303702031D59293E1859293E14B11750
:1002B000912202303702031D6229BE186229BE1442
:1002C000B117932203303702031D6B293E196B29A6
:1002D0003E15B117952204303702031D7429BE194B
:1002E0007429BE15B117992225082F02031D9D29D7
:1002F00001303702031D81293E1C81293E10B117B0
:100300009D2202303702031D8A29BE1C8A29BE1095
:10031000B1179F2203303702031D93293E1D9329F5
:100320003E11B117A12204303702031D9C29BE1DC6
:100330009C29BE11B117A5229D29B70A05303702A5
:1003400003180800FA28B601B3019630B400013052
:10035000B5000130B70085018701B1131D22B2201D
:10036000B30BD529031085190314BA0DF0303A02E6
:1003700003190D2AB40BD529013037020319A9221C
:10038000023037020319AD22033037020319B122BC
:10039000043037020319B5223708B6080319B6002E
:1003A0000319D329B6039630B400311DAF2931119A
:1003B000321CDF292D090339AD00AE09AF095130D8
:1003C0002F0655390319F42905302F06553903191D
:1003D000F42915302F0655390319F42955302F0605
:1003E00055390319F429AF29AF13AF12AF11AF106C
:1003F0008B1320303707BC002F08BB005B22103066
:100400003707BC002E08BB005B2200303707BC005A
:100410002D08BB005B228B17172285018701B70AC5
:10042000B60105303702031CAF29B9220800043099
:10043000370203190800850187016430B9003330A1
:100440000F1E85000F1A8501FF300F1A87000F1E3F
:100450008701B220311D1F2A3111321C342A2D0987
:100460000339AD00AE09AF0951302F0655390319D4
:100470001D2A05302F06553903191D2A15302F0660
:10048000553903191D2A55302F06553903191D2AD0
:10049000B90B1F2A850187010800B11F0800B1139D
:1004A0001030BC003E08BB005B223030BC003F086F
:1004B000BB005B2208003C088B1383169B001C14B6
:1004C0001A0883128B173B02031908008B133B0891
:1004D00083161C159A0083123C0883169B00553026
:1004E0009D00AA309D009C1464009C18742A1C1165
:1004F00083128B170800831600309B001C141A0807
:100500008312BD00831610309B001C141A0883123E
:10051000BE00831630309B001C141A088312BF00E3
:1005200008008516080005160800BD180800851487
:100530000800BD18080005140800851208000512FF
:100540000800BD18080085100800BD180800051037
:1005500008000508203A850008000508103A8500C3
:1005600008000508023A850008000508013A8500E0
:1005700008003E188516BE180516BD1808003E195D
:100580008514BE1905140800B601B301B4013D1C61
:10059000CC2A3D10BD14CF2AC030BD053D143D0806
:1005A0003F39B6006400D42AD52AD62AD72AD82AB9
:1005B0003330B41B8500B41F8501B30BD22AB40BB2
:1005C000D22A0310B60CB608031DD22A0030BC0094
:1005D0003D08BB005B220800BF1FF72A3F1B8510A8
:1005E0003F1B05143F1F85143F1F05100800851091
:0605F000051008000800E0
:084000000500000006000200AB
:02400E00CC33B1
:10420000010003000300030003000200020002009B
:10421000020000000000FF00FF00FF00FF00FF00A1
:10422000000000000000000000000000000000008E
:104230000000C000C000FF00FF00FF00FF00FF0003
:104240000100510005001500550051000500150042
:10425000550051000500FF00FF00FF00FF00FF00B8
:104260000000FF00FF00FF00FF00FF00FF00FF0055
:10427000FF00FF00FF00FF00FF00FF00FF00FF0046
:10428000FF00FF00FF00FF00FF00FF00FF00FF0036
:10429000FF00FF00FF00FF00FF00FF00FF00FF0026
:1042A000FF00FF00FF00FF00FF00FF00FF00FF0016
:1042B000FF00FF00FF00FF00FF00FF00FF00FF0006
:1042C000FF00FF00FF00FF00FF00FF00FF00FF00F6
:1042D000FF00FF00FF00FF00FF00FF00FF00FF00E6
:1042E000FF00FF00FF00FF00FF00FF00FF00FF00D6
:1042F000FF00FF00FF00FF00FF00FF00FF00AA001B
:00000001FF
